:1000000004EE00F011EE00F00EEC00F00FEE70F0D8
:1000100010EE0FF00EEC00F0D2EF3FF0EE6AE5507C
:0A002000E150FCE1E250FAE11200A9
:107F66000001FF6F000E00010001FE6F0001FF51CE
:107F76000BD04E0E0001FF6FD30EE82EFED7FF2F5B
:107F8600FCD700010001FE2B00010001FD5100019C
:107F96000001FE5DD8A001D001D0EBD71200000190
:107FA600FC6F640E00010001FB6F0001FC51FD0E29
:107FB600936E81A801D001D009D00001FC6F640E38
:107FC60000010001FB6F0001FC5108D00001FC6FAD
:107FD6000F0E00010001FB6F0001FC51020E8A6EBC
:107FE600FBC0FDF0B3EC3FF0000E8A6EFBC0FDF067
:0A7FF600B3EC3FF0DED700EF00F01F
:020000040030CA
:08000000240F000000818100C3
:00000001FF
